:020000040000FA
:0400000000001028C4
:08000800F1000308F2000A08F0
:10001000F30073088A0072088300F10E710E090064
:10002000860183160313811307178717A0308700F3
:100030007F308600FF3085008312AA273C30850080
:10004000B501A601D301DA01DB01DC01DE01EE011D
:10005000B801A701D001A801D101A901AA01AB01F2
:10006000AC01C601D201DF01C501E901ED01CF01FB
:100070000230CB000712F601F7011E30DD001C3004
:10008000E30064308E2708308A00052000308A00A3
:10009000D2164F10CF14CF164F11CF114F124F134E
:1000A0005211CF1952154F1B52154611DF17D21797
:1000B000A9170B108B15FF30F800F9006430FA0017
:1000C000D10AD10B64285213C61F6C285A08D100DC
:1000D000DA016221C6136028AD20B520E726291871
:1000E00072288928CF1C7B28A91A7B28A9187F2869
:1000F00010309E277F28452626080A261926A91F84
:1001000088282608C03EB4275F2410309E27602828
:100110005B218425C000C01BAA28401C9E28A91F63
:1001200096286508C03EB4275F2460285B215F10D5
:10013000D30AD30B9D285F146028C513C01CA128C7
:10014000BD28401DA428D728C01D60286508B427F5
:100150005F2460284619C32760285F1C0800C51B60
:100160000800FD30B427C5170800DF1C0800451B38
:100170000800FD30B427451708006508C0000830A6
:10018000E90040080339E907C00DC00D4008F03907
:10019000E907EC018030B4276908B4276708B42761
:1001A0006808B4276C08B427FF30B42760280830EB
:1001B000E900E701E8016708EC00CA28452600309D
:1001C0000A261926C51008002C1876292C1976291C
:1001D000AC1A76292C1B7629CF1DF4284F1E7629C0
:1001E0002808073A03191029C61D76292808053A58
:1001F0000319182928080D3A03191D292808153A4A
:10020000031926292808253A03192F2928081D3AF9
:10021000031936292808353A03193B292808762975
:100220002F30562164309E27521339305621080052
:1002300014305621083056210800013056210E3066
:1002400056210430562132305621080014305621F0
:1002500008305621053056213230562108000F3023
:1002600056210630562132305621080001305621E1
:10027000323056210800143056210F3056213230CA
:1002800056210800C613CC008024C40AC40B4D2993
:1002900032305621D101DA01080044085621CC0A37
:1002A0002A083B3A031D55292C164429AA0003307D
:1002B0009E275213902B08308A001B2001308A00A1
:1002C000291E08005108003A031908005108A80027
:1002D000A91E702909308A00B22101308A00080065
:1002E0002808B327C619E4284F1AE428C51E7C291C
:1002F0007608F7002808F600CF1D80294F1E2F2B07
:10030000DA0ADA0B84292F2B51086624AA005A082E
:100310006624C700DF1B2F2B1F302A0203189529E4
:100320001F3047020318B1292F2B2A08C4001E30A2
:10033000C402CD21C41F2F2B441BAA294418FF2916
:10034000C418122A4419252AC419382A441AEC2937
:10035000C41AD92944184B2AC4185E2A4419712A90
:100360002F2B4708C4001E30C402CD21C41F2F2BE1
:10037000441BC6294418AA2AC418BD2A4419D02AE5
:10038000C419E32A441A972AC41A842A4418F62A5C
:10039000C418092B44191C2B2F2B0030C407103014
:1003A0000318013E8A0044080020C40001308A007E
:1003B00008000130C2002330C70710300318013E87
:1003C0008A0047082320C40001308A00C40AC40BF5
:1003D000EA298E2B440842290130C2007B30C7072E
:1003E00010300318013E8A0047087B20C40001300A
:1003F0008A00C40AC40BFD298E2B4408422901300F
:10040000C200D330C70710300318013E8A004708E6
:10041000D320C40001308A00C40AC40B102A8E2BDA
:10042000440842290230C2002B30C707113003189C
:10043000013E8A0047082B21C40002308A00C40A0A
:10044000C40B232A8E2B440842290230C200DB3021
:10045000C70711300318013E8A004708DB21C4009A
:1004600002308A00C40AC40B362A8E2B4408422963
:100470000230C2008330C70711300318013E8A00E2
:1004800047088321C40002308A00C40AC40B492AE9
:100490008E2B440842290430C2003330C707123083
:1004A0000318013E8A0047083322C40002308A0044
:1004B000C40AC40B5C2A8E2B440842290430C200B3
:1004C0008B30C70712300318013E8A0047088B2281
:1004D000C40002308A00C40AC40B6F2A8E2B440861
:1004E00042290430C200E330C70712300318013E2E
:1004F0008A004708E322C40002308A00C40AC40B01
:10050000822A8E2B440842290130C2004F30AA07AC
:1005100010300318013E8A002A084F20C400023020
:100520008A00C40AC40B952A8E2B44084229013044
:10053000C200A730AA0710300318013E8A002A081B
:10054000A720C40002308A00C40AC40BA82A8E2B3C
:10055000440842290130C200FF30AA0710300318B6
:10056000013E8A002A08FF20C40002308A00C40A23
:10057000C40BBB2A8E2B440842290230C2005730DC
:10058000AA0711300318013E8A002A085721C40027
:1005900002308A00C40AC40BCE2A8E2B440842299A
:1005A0000230C2000730AA0712300318013E8A0049
:1005B0002A080722C40002308A00C40AC40BE12AB8
:1005C0008E2B440842290230C200AF30AA071130F6
:1005D0000318013E8A002A08AF21C40002308A00B5
:1005E000C40AC40BF42A8E2B440842290430C200EA
:1005F0005F30AA0712300318013E8A002A085F22E2
:10060000C40002308A00C40AC40B072B8E2B440896
:1006100042290430C200B730AA0712300318013E45
:100620008A002A08B722C40003308A00C40AC40B17
:100630001A2B8E2B440842290430C2000F30AA071F
:1006400013300318013E8A002A080F23C400033028
:100650008A00C40AC40B2D2B8E2B4408422928087B
:100660003F3A0319EC2C28082D3A0319062D2808C7
:10067000123A03191E2D28082F3A0319422D280873
:10068000373A0319502D28083B3A031D8E2B4F1281
:10069000CF195215C51E8E2B7708043A031D572B10
:1006A0004F14CF10CF124F11CF114F138D2B77084E
:1006B0001A3A031D622B4F10CF14CF124F15CF11D2
:1006C0004F138D2B7708323A031D6D2B4F10CF142B
:1006D000CF124F11CF154F138D2B7708183A031DEA
:1006E000782B4F10CF14CF164F11CF114F138D2BE6
:1006F00077080E3A031D832B4F10CF14CF124F11E2
:10070000CF114F178D2B7708163A031D8D2B4F10E5
:10071000CF14CF124F15CF114F13C5126524AA0065
:10072000AB01521F9E2B1F302A02031C9E2B2A084E
:10073000323A03199E2BD21B9E2B080052172C1CF9
:10074000AE2B3F30AB002C1DBB2B0030AB001F305D
:100750002A02031CBB2B7E30AB00BB2B2C1DB32B02
:100760007E30AB00BB2B1F302A020318BB2B2C1E84
:10077000BB2BBD30AB002A08AB0774242D085219DF
:10078000803EB4275F24CF18CC2B451E5A25451236
:1007900008004516AD00BE2B4F19FF2BCF19E92BD2
:1007A000CF1AD82B4F1B0B2C451E5A25451208007B
:1007B00045262D08C0000830F5000D260330C00086
:1007C0000330F5000D2607309E27451E5A25451299
:1007D00008004F1AEF2B52102D08B624F82B521494
:1007E0002D08A8241F302D020318F82B2C1AEF1205
:1007F0000230CB002324451E5A25451208003C3008
:10080000C726F030C7262D08C72603309E27451E71
:100810005A25451208002D08C4246F08FF3A031911
:100820001D2C6F08D1240030BF00033078260E3015
:100830009E270330BF006F0878260E309E27451E86
:100840005A25451208006F08FF3A0319532C2D084A
:10085000323A031D302C4F1E462C2030EF00462C20
:100860002D08C0002A3040020318372C462C2D08D2
:10087000C0004030400203183F2C5210462C2D0877
:10088000C0006A30400203185210462CA9184C2CA4
:1008900032309E2718309E2729266F08D825E72555
:1008A000CB0B4A2CCB0A28080E3A03194F162808FE
:1008B0001F3A03194F1252154F1A52110800FF30F8
:1008C000F800F9006430FA0008002808C40000307D
:1008D000C40718300318013E8A0044080020C400F1
:1008E00004308A00440808000030AB0719300318B0
:1008F000013E8A002B080021AD0004308A00080068
:10090000C218902C42199C2C0030CC071C300318C4
:10091000013E8A004C080024C40004308A0008000C
:100920000030CC071D300318013E8A004C0800251A
:10093000C40004308A0008000030CC071E300318C1
:10094000013E8A004C080026C40004308A000800DA
:100950002D08C0000030C0071A300318013E8A007D
:1009600040080022EF0004308A0008002D08C00073
:100970008130C0071A300318013E8A0040088122E6
:10098000EF0004308A000800C0000030C0071B30B0
:100990000318013E8A0040080023EF0004308A005B
:1009A0000800C0004230C00718300318013E8A001A
:1009B00040084220EF0004308A0008002C1808008C
:1009C0002C190800AC1A0800AC132C13C61DEA2C15
:1009D000C6110800C61508003D30C923A9122C1BFA
:1009E000DE2C2C1EFC2CAC19FC2C2C12AC13BB30B6
:1009F000D21FC923A91608002C1C002D2C1008009A
:100A00002C1408007930C9235A2508007E30C923E8
:100A10002C1B1A2D2C1E0F2DAC190F2D022D2C1D49
:100A2000162DAC1C182D2C11AC1008002C1508002C
:100A3000AC1408007A30C9235A250800BC30D21BF8
:100A4000C923AC19372DAC1B302D2C1E3D2D2C1677
:100A5000AC15BB30D21FC9237730D21FC923080081
:100A6000AC132C12AC11BB30D21FC92308002C12BE
:100A7000AC11F730D21FC92308002C163B30D21F0F
:100A8000C9230800AC1E482DAC12BE30C923080093
:100A90002C19C516CF19C516AC163E30C92308004F
:100AA0002C1F562D2C13BF30C92308002C173F30A4
:100AB000C9230800AC1E5F2DAC12BE30C9232C1F09
:100AC000642D2C13BF30C923AC18692D2C1D692D42
:100AD0002C11AC1908002C1E08002A302A02031C15
:100AE0007F2D2A08353C031C7F2D32302A0603193E
:100AF0007F2D2E302A0603197F2DAC1708002C12EB
:100B0000BB30D21FC9230800061BD62D0B27003A85
:100B1000031DD62DE5013727003A031DD62D4008C9
:100B2000E500E601E701E8014627003A031DD62D5E
:100B30004008E600631266081C396306031DA62DF3
:100B400066186517E618E517631608346316660815
:100B50001C396306031DD62DE61CB12D6508D30094
:100B6000013457274518D62D57274518D62D803ADA
:100B70000319CB2D1D27003A031DD62D4008E70091
:100B80001D27003A031DD62D4008E8007C27003AB7
:100B9000031DD62D02341D27003A031DD62D400813
:100BA000E7007C27003A031DD62D04348034280842
:100BB000C0000730F500401CE22D4A26C00CF50BA2
:100BC000DB2D08003326C00CF50BDB2D0800521C72
:100BD000F42D0530F5001A30C000F8250830F50076
:100BE0006130C000F82508000530F5000F30C00066
:100BF000401CFF2D2E26C00CF50BF82D08003326C7
:100C0000C00CF50BF82D0800C0000830F5000D26CB
:100C100008002808C0000630F500401C142E4A26A3
:100C2000C00CF50B0D2E08004F26C00CF50B0D2E39
:100C300008001E30C0000530F500401C242E4A2656
:100C4000C00CF50B1D2E08004F26C00CF50B1D2EF9
:100C5000080007106A265730F4003C2E07106A2659
:100C60003030F4003C2E07106A2601309A27382EC7
:100C700000001930F4003C2E071402309A270710A8
:100C800001309A27F40B3C2E0800071062264E30E4
:100C9000F400572E071062262B30F400572E071051
:100CA000622601309A27542E1630F400572E07146E
:100CB00002309A270000071001309A275F2EF40BAC
:100CC000572E080031309A2731309A2724309A273E
:100CD000692E080031309A2731309A2727309A2719
:100CE0000800C000871402309E27871002309E271C
:100CF000C0001230BB265A30AF261230BB26461435
:100D00000830F50089263F08C0000830F500892624
:100D10000800401C902EA426C00CF50B892E08005C
:100D20009526C00CF50B892E080046189E2E000053
:100D30001230BB261130AF26000008001230AF265B
:100D40001130BB26000008004618AB2E00002530ED
:100D5000BB26461408002530AF2646100800F400D4
:100D6000071002309A270000000001309A27B82EA1
:100D7000F40BB02E0800F400071402309A2700008C
:100D8000071001309A27C42EF40BBC2E0800C000B7
:100D9000DF260830F500401CD32ED926C00CF50BF9
:100DA000CB2ED9260800DF26C00CF50BCB2ED9267A
:100DB0000800071016309A27DD2E000008000714DF
:100DC00004309A27071011309A27E62E0800A70151
:100DD000D3012910C90B08001930C900CA0B08003B
:100DE0001930CA000608FF3A3F39A600A7000030B4
:100DF0002606031D032FDF14D301B80AB80B03190D
:100E00000800B803072FDF1045132030B80026086C
:100E1000D30029140800871329131030B900061BCA
:100E2000EE3418309A27B90B0F2F061F152F4330B9
:100E30009A271A2F000087170034C0010830BA0023
:100E4000C00CC01357274518EE34C007BA0B202F2B
:100E500040080034C0010730BA0057274518EE3467
:100E6000C007C00CC013BA0B2D2F40080034C001BE
:100E70000630BA0057274518EE34C007C00CC0131F
:100E8000BA0B3A2FC00CC01340080034C001053023
:100E9000BA0057274518EE34C007C00CC013BA0B70
:100EA000492FC00CC013C00CC013400800344510BB
:100EB0001D30B900061B632F01309A275F2FB90B35
:100EC0005A2F4514080087173630B90001309A2789
:100ED000692F061F6F2FB90B662F45140800871363
:100EE0004630B90001309A27752FB90B722F87173A
:100EF000061F7B2F00348034061F7C2F5430B9002E
:100F0000061F882F01309A27852FB90B802F0034B8
:100F1000EE3408000800080008000800AF00643044
:100F2000B0002030B100B10B932FB00B912FAF0B5D
:100F30008F2F0800FF3E031D9A2F0800AF000A30D4
:100F4000B0002030B100B10BA32FB00BA12FAF0B1D
:100F50009F2F0800831619309900243098008312BF
:100F600080309800080008000C1EB42F990008007B
:100F70006508B3276608B3276708B3276808B3274F
:100F8000DB30B3270800F80B0800FF30F800F90B3E
:100F90000800FF30F900FA0B08006430FA0007116E
:100FA00087110712FF309E27FF309E2783160313F9
:100FB0003F3086008312FF309E27FF309E27FF3090
:100FC0009E27FF309E270B1063000000831603133B
:100FD0007F308600831206080B10FF309E27071211
:0A0FE000F601F701FF309E2708001C
:1010000008000C1E012899000800473000204B30D2
:1010100000204F300020533000200D300020080009
:101020001E30A91A0730DD00A91005308A005A25A4
:1010300008308A00080029125E08D100D30AD30BB9
:1010400022282F285308C4005B084402031D2F28C0
:10105000DD0B2F28DD0A2916A91452133128A918EF
:101060001020531C3628D40AD40BD403D31C3B289D
:10107000D50AD50BD503531D4028D60AD60BD60367
:10108000D31D4528D70AD70BD703531E4A28D80AA1
:10109000D80BD803D31E4F28D90AD90BD903EE0A8F
:1010A000EE0B53285528EE0366285308C4005B084E
:1010B000C406C4050319662829160530EE00D215AA
:1010C00052121E30A91A0730DD00A9105C08C400B6
:1010D0005B08C406C405031D52165B08DE005308F6
:1010E000DE05291E8829C801C613A001A101A2019D
:1010F0007F30A300A400A500D11E83282030A000CB
:101100005908A300A628511E8A281030A0005808AC
:10111000A300AD28D11D91280830A0005708A300D6
:10112000B428511D98280430A0005608A300BB28FD
:10113000D11C9F280230A0005508A300C228511CD2
:10114000E4280130A0005408A300E428511EAD2873
:101150001030A1005808A400C928D11DB4280830B7
:10116000A1005708A400D028511DBB280430A100BD
:101170005608A400D728D11CC2280230A100550867
:10118000A400DE28511CE4280130A1005408A4006A
:10119000E428D11DD0280830A2005708A500E42873
:1011A000511DD7280430A2005608A500E428D11C00
:1011B000DE280230A2005508A500E428511CE428CE
:1011C0000130A2005408A500FF30002023087F3C16
:1011D000A300002024087F3CA400002025087F3CB9
:1011E000A50000202308003A031901292408003A29
:1011F00003190C29240823020319012903180129C2
:101200000C292508003A031934292508240203195A
:1012100051290318512934292508003A031917299F
:101220002508230203191729031851291729230810
:10123000C300EE00EE0CEE13EE01EE146E1404305B
:1012400043020318C30323082402430203182B2973
:10125000C6172108C80023082502430203186D2978
:10126000C6172208C8076D292408C300EE00EE0C3B
:10127000EE13EE01EE146E14043043020318C303A0
:1012800024082302430203184829C6172008C8006F
:1012900024082502430203186D29C6172208C8072F
:1012A0006D292508C300EE00EE0CEE13EE01EE14DE
:1012B0006E14043043020318C303250824024302BA
:1012C00003186529C6172108C80025082302430210
:1012D00003186D29C6172008C807D21A7129C6132A
:1012E0007929C61F79295108C400DA004808D100BD
:1012F0007B295108C4007F304418D400C418D5009D
:101300004419D600C419D700441AD800C41AD90009
:101310005B08DC005308DB007F30531CD400D31C77
:10132000D500531DD600D31DD700531ED800D31EA1
:10133000D9000800AF000A30B0002030B100B10B76
:101340009F29B00B9D29AF0B9B290800C40080305A
:101350000120440801200800012000300120FF3056
:10136000012008003F302806031DBD29A912323094
:101370008E27DB01DC01DE0108003F302806031D5B
:10138000C229A9122808093A0319312A28081B3A48
:101390000319392A2808083A0319412A2808193A52
:1013A0000319492A2808183A0319492A2808103A23
:1013B0000319592A2808383A0319612A2808303AAB
:1013C0000319792A2808203A0319712A2808343A7F
:1013D0000319792A2808243A0319812A2808363A59
:1013E0000319892A2808043A0319912A2808263A59
:1013F0000319992A2808063A0319992A2808023A53
:101400000319A92A2808073A0319B12A2808033A18
:101410000319C92A2808013A0319C12A28080B3AD6
:101420000319C92AA918080028083B3A0319D12A28
:1014300028081F3A0319F92A2808053A0319D12A5E
:101440002808283A0319F92A2808123A0319D12A38
:1014500028082D3A0319E32A28080C3A03190B2B04
:1014600008006D08083EA6210030AA210530AC21F5
:1014700008006D08083EA6210030AA210F30AC21DB
:1014800008006D08083EA6210330AA210330AC21D4
:1014900008006D08083EA6210A30AA210A30AC21B6
:1014A00008006D08083EA6210430AA210230AC21B4
:1014B00008006D08083EA6210530AA210030AC21A5
:1014C00008006D08083EA6210F30AA210030AC218B
:1014D00008006D08283EA6210430AA21FE30AC2168
:1014E00008006D08283EA6210330AA21FD30AC215A
:1014F00008006D08283EA6210A30AA21F630AC214A
:1015000008006D08283EA6210030AA21FB30AC213E
:1015100008006D08283EA6210030AA21F030AC2139
:1015200008006D08383EA621FD30AA21FD30AC210F
:1015300008006D08383EA621F630AA21F630AC210D
:1015400008006D08383EA621FC30AA21FE30AC21EF
:1015500008006D08183EA621FB30AA210030AC21FE
:1015600008006D08183EA621F030AA210030AC21F9
:1015700008006D08183EA621FC30AA210230AC21DB
:1015800008006D08183EA621FC30AA210430AC21C9
:1015900008006D08183EA621F630AA210A30AC21B9
:1015A00008001E308E270930A6210030AA21003005
:1015B000AC210130ED000830A6210030AA21003016
:1015C000AC21ED01B9291E308E270930A62100304B
:1015D000AA210030AC210130ED00B92932308E272C
:1015E0000C30A6210030AA210030AC210430ED00DF
:1015F000B92932308E270A30A6210030AA210030C6
:10160000AC210130ED000830A6210030AA210030C5
:10161000AC21ED01B92932308E270830A6210030E7
:0A162000AA210030AC21ED01B92928
:10200000820081348234843488349034A0340034A3
:102010000034003400340034C134C234003400349D
:102020000034003400340034003400340034003410
:1020300000340034003400340034C434003400343C
:1020400000340034080082000034003400340034CE
:1020500000340034003400340534003400340034DB
:1020600000340034003401340034003400340834C7
:1020700000340034003400340D34003400340034B3
:1020800000340034003400340034003400340034B0
:102090000034003400340034003400340034820052
:1020A000003411340034153400340034003400346A
:1020B0000034003400340034003400340034003480
:1020C0000034003400340034003400340034003470
:1020D0000034003400340034003400340034003460
:1020E0000034003400340034003400340034003450
:1020F00000340034003482000034003400340034F2
:102100000034003400341E340034003400342134F0
:102110000034003400340034183400340034003407
:10212000003400340034003400340034003400340F
:1021300026340034003400340034003400340034D9
:1021400000340034003400340034003400348200A1
:102150002B340034003400342E3400340034003486
:1021600000340034003400340034003400340034CF
:1021700000340034003400340034003400340034BF
:1021800000340034003400340034003400340034AF
:10219000003400340034003400340034003400349F
:1021A0000034003400348200003400340034003441
:1021B000003400340034003400340034003400347F
:1021C000393400340034003400343E3400340034F8
:1021D00000343434003400344434003400340034E7
:1021E000003400340034003400340034003400344F
:1021F00000340034003400340034003400348200F1
:10220000003448340034003400344D340034003499
:10221000003400340034003400340034003400341E
:10222000003400340034003400340034003400340E
:1022300000340034003400340034003400340034FE
:1022400000340034003400340034003400340034EE
:102250000034003400348200003400340034003490
:1022600000340034003400340034073400340034C7
:1022700000340434003400340034003400340034BA
:1022800001340034003400340034003400340034AD
:102290000F3400340034003400340034003400348F
:1022A0000034003400340034003400340034820040
:1022B0000034003415340034593400340034003410
:1022C000003400340034003400340034003400346E
:1022D000003400340034003400340034003400345E
:1022E000003400340034003400340034003400344E
:1022F000003400340034003400340034003400343E
:1023000000340034003482000034003400340034DF
:1023100000340034003400340034003400342334FA
:10232000003400340034003400341F3400340034EE
:1023300000340034003428340034003400340034D5
:1023400000343034003400340034003400340034BD
:10235000003400340034003400340034003482008F
:102360003434003400340034003438340034003461
:1023700000340034003400340034003400340034BD
:1023800000340034003400340034003400340034AD
:10239000003400340034003400340034003400349D
:1023A000003400340034003400340034003400348D
:1023B000003400340034820000340034003400342F
:1023C000003400340034003400344234003400342B
:1023D00000340034003400340034003400343E341F
:1023E000003400340034003400344B3400344734BB
:1023F000003400340034003400340034003400343D
:1024000000340034003400340034003400348200DE
:10241000003400344E34533400340034003400347B
:10242000003400340034003400340034003400340C
:1024300000340034003400340034003400340034FC
:1024400000340034003400340034003400340034EC
:1024500000340034003400340034003400340034DC
:10246000003400340034820000340034003400347E
:1024700000340034003408340034003400340034B4
:1024800000340034003401340034003400340034AB
:102490000034003400340D3400340034003414347B
:1024A000003400340034003400340034003400348C
:1024B000003400340034003400340034003482002E
:1024C0001734003400341A3400340034003400343B
:1024D000003400340034003400340034003400345C
:1024E000003400340034003400340034003400344C
:1024F000003400340034003400340034003400343C
:10250000003400340034003400340034003400342B
:1025100000340034003482000034003400340034CD
:10252000003400340034003400340034003400340B
:1025300000342734003400340034003400340034D4
:102540000034213400340034003431340034003499
:1025500000342B34003400340034003400340034B0
:10256000003400340034003400340034003482007D
:10257000003400343634003400343D340034003448
:1025800000340034003400340034003400340034AB
:10259000003400340034003400340034003400349B
:1025A000003400340034003400340034003400348B
:1025B000003400340034003400340034003400347B
:1025C000003400340034820000340034003400341D
:1025D00000340034003400344A3400340034003411
:1025E00051340034003400344134003400340034B9
:1025F0004E340034003400340034003400340034ED
:10260000003400340034003400340034003400342A
:1026100000340034003400340034003400348200CC
:10262000003454340034003457340034003400345F
:1026300000340034003400340034003400340034FA
:1026400000340034003400340034003400340034EA
:1026500000340034003400340034003400340034DA
:1026600000340034003400340034003400340034CA
:06267000003400340034C8
:103000008200013402340F3403341B3413342E3461
:1030100004342A342434103421341C3414342F342E
:10302000053423343B34113420341D34153430340A
:103030000734083409342C340A342934263438341B
:10304000063422341F3412342B341E3416343134F7
:103050001734183419343A341A343C3428343E3492
:103060000B340C340D3425340E3427342D343F34D6
:1030700032343334343436343534373439343D34FF
:103080000034003482001534133410343B343834A7
:103090000034003479340034003400340034003417
:1030A0000034003400340034003400340034003480
:1030B0000034003400340034003400340034003470
:1030C000003400341634543457340034003400349F
:1030D000003400340034003400341C340034003434
:1030E0000034003400340034003402340734043433
:1030F0000D340E340B34083419341A3401341F34AF
:063100000034003400342D
:1032000082000134023403340434053406340734B4
:10321000083409340A340B340C340D340E340F34B2
:103220001034113412341334143415341634173462
:10323000183419341A341B341C341D341E341F3412
:1032400020342134223423342434253426342734C2
:10325000283429342A342B342C342D342E342F3472
:103260003034313432343334343435343634373422
:10327000383439343A343B343C343D343E343F34D2
:103280004034413442344334443445344634473482
:10329000483449344A344B344C344D344E344F3432
:1032A00050345134523453345434553456345734E2
:1032B000583459345A345B345C345D341F34203410
:1032C000213422342334243425342634273428343A
:1032D00029342A342B342C342D342E342F343034EA
:1032E000313432343334343435343634373438349A
:1032F00039343A343B343C343D343E343F3440344A
:1033000041344234433444344534463447344834F9
:1033100049344A344B344C344D344E344F345034A9
:103320005134523453345434553456345734583459
:1033300059345A345B345C345D345E345F34603409
:1033400061346234633464346534663467346834B9
:103350002A342B342C342D342E342F343034313461
:103360003234333434343534363437343834393411
:103370003A343B343C343D343E343F34013402343F
:1033800003340434053406340734083409340A3469
:103390000B340C340D340E340F3410341134123419
:1033A00013341434153416341734183419341A34C9
:0833B0001B341C341D341E34D3
:103400008200613462346334643465346634673412
:10341000683469346A346B346C346D346E346F34B0
:103420007034713472347334743475347634773460
:10343000783479347A347534613461346F342E34AD
:103440002C3421343F342D3427345C342F34203451
:103450007E345E34FF341D34163415342B342B3453
:103460002B342B344C342C342C342C343C34183442
:10347000FF340F34FF34FF34FF34FF34FF34FF34A4
:103480003134323433343434353436343034373400
:10349000383439340A34203426340A342B34253471
:1034A000203420342A34203424342034283428345E
:1034B0003C342934293429343E3429343A343B34D9
:1034C00020342034203422342A342A342034203446
:1034D00020342034FF34FF34FF34FF34FF34FF3412
:1034E000FF34FF34FF34FF34FF34FF34FF34FF3444
:1034F000FF34FF34FF34FF34FF34FF34FF34FF3434
:10350000FF348200FF342034FF34FF342134FF3491
:10351000FF341E34FF34FF340A3419341F340A34A4
:1035200029342934FF342D3419343C34FF34FF342A
:103530002C34FF341834FF342B34FF34FF34FF3481
:10354000FF34FF34FF34FF34FF34FF34FF34FF34E3
:10355000FF34FF34FF34FF341D341634153428345F
:10356000203420342B342A34213421342C343B347D
:10357000183428340F34FF34FF34FF34FF34FF3461
:10358000FF34003401340234033404340534093484
:103590000634073408340A34FF34FF34FF34FF3470
:1035A000FF34FF34FF34FF34FF34FF34FF34FF3483
:1035B000FF34FF34FF34FF34FF34FF34FF34FF3473
:1035C000FF34FF34FF34FF34FF34FF34FF34FF3463
:1035D000FF34FF34FF34FF34FF34FF34FF34FF3453
:1035E000FF34FF34FF34FF34FF34FF34FF34FF3443
:1035F000FF34FF34FF34FF34FF34FF34FF34FF3433
:103600008200043424340534023423340334FF3478
:10361000FF34FF34FF340A3419341F340A34293498
:103620002934FF342D3419343C34FF34FF342C3426
:10363000FF341834FF342B34FF34FF34FF34FF34AD
:10364000FF34FF34FF34FF34FF34FF34FF34FF34E2
:10365000FF34FF34FF341D34163401342834203451
:1036600020342B342A34213421342C343B34183484
:1036700028340F34FF34FF34FF34FF34FF34FF3479
:10368000003401340234033404340534093406347C
:10369000073408340A34FF34FF34FF34FF34FF3476
:1036A000FF34FF34FF34FF34FF34FF34FF34FF3482
:1036B000FF34FF34FF34FF34FF34FF34FF34FF3472
:1036C000FF34FF34FF34FF34FF34FF34FF34FF3462
:1036D000FF34FF34FF34FF34FF34FF34FF34FF3452
:1036E000FF34FF34FF34FF34FF34FF34FF34FF3442
:1036F000FF34FF34FF34FF34FF34FF34FF34FF3432
:103800008200103415341434003409341334003475
:103810001434083401341434003419340F3415349A
:103820000034023415341434003404340F340034BA
:103830001134153409341434053400340834053493
:1038400000340C3409340B34053400341434083497
:1038500005341934003401340D3400340534013496
:103860000334083400340034163405341234193467
:1038700000340D3415340334083400341234093460
:103880000734083414340034193405341334003444
:103890000234053405340E340034063412340F3447
:1038A0000D3400340034003400340034003400346B
:1038B0000034003400340034003400340034003468
:1038C0000034003400340034003400340034003458
:1038D0000034003400340034003400340034003448
:1038E0000034003400340034003400340034003438
:0E38F00000340034003400340034003400345E
:103A000082001534103400340E340F340034033483
:103A1000053412341434013409340E3400341434AF
:103A20000834053412340534003403340F340D34B3
:103A300005340034003400340034003400340134E0
:103A40001234053400340C340F340E34073400348F
:103A50000534183401340D3410340C34053400347A
:103A60000F3406340634003401340C340C34003482
:103A700006340934123413341434003414340F343B
:103A80000F3400340A341534133414340034013440
:103A90000E3419340034173405340034033401343F
:103AA0000D340534003404340F340E34243414340B
:103AB000003405341634053412341934003400341B
:103AC0000034003400340034003400340034003456
:103AD0000034003400340034003400340034003446
:103AE0000034003400340034003400340034003436
:103AF0000034003400340034003400340034003426
:103C00008200103405340F3410340C340534003481
:103C100008340134163405340034053418340334C0
:103C2000153413340534003401340E3400340134B7
:103C30001434003404341534123409340E34073487
:103C400000341634093413340934143400340E3477
:103C50000F34143400340F340634143405340E3465
:103C600000341734083405340E3400340334083477
:103C700001340E3407340534003406340F34123462
:103C800000341134153405341334143409340F342A
:103C90000E3400343B34093400340034153413340A
:103CA00000340D3405340034023405340034053456
:103CB000163405340E34003400340034003400343B
:103CC0000034003400340034003400340034003454
:103CD0000034003400340034003400340034003444
:103CE0000034003400340034003400340034003434
:103CF0000034003400340034003400340034003424
:02400E00313F40
:00000001FF
